:1000000029C036C035C034C033C032C031C030C062
:100010002FC02EC0798D9AA2AAFFA3A3A3A1A1A14C
:10002000A1A1A1A3A3A3A3A3A1A1A1A1A114E6FFA0
:10003000000000000002146EFFFFFF00000000003F
:1000400000005AFFFCFEFDFF000000073889FFFC9E
:10005000FEFDFF0011241FBECFE9CDBF10E0A0E6DA
:10006000B0E001C01D92AC36B107E1F7D0D0BBC102
:10007000C7CF26EB33E003C0F9013197F1F70197C1
:10008000D8F7089588EE93E0F4CFCF93C091630042
:100090008C2F8F5F8F738093630090916100929596
:1000A000990F907E609162006295660F660F607C8A
:1000B000692B90916000692B90E087D16FEF8C2FB6
:1000C00090E0CF9182C1CF931092630008C08C2F33
:1000D00090E073D18F3F41F4CF5FC0936300C09134
:1000E0006300C034A0F30EC0982F9F7090936000FF
:1000F00085FB992790F99093610086FB882780F90A
:1001000080936200CF91089580916100811112C0A7
:1001100087E08093660088E490E090936A00809383
:10012000690085E390E0909368008093670082E225
:1001300090E011C084E08093660080E490E09093AA
:100140006A00809369008DE290E09093680080934C
:1001500067008AE190E0909365008093640080914D
:1001600066008C5F80936B000895811104C061115B
:1001700002C091EA9FBD89BD66BF089590E0E091FD
:100180006400F0916500E80FF91FE491EFBDE09184
:100190006700F0916800E80FF91F6491E091690031
:1001A000F0916A00E80FF91F8491DFCF369A3699F3
:1001B000FECF85B108951F93CF93DF93C82F14E12D
:1001C000D1EA0CC019BC16BF84E690E052DFDFBD57
:1001D00019BC16BE80E991E04CDFC150C111F2CFCD
:1001E000DF91CF911F9108951F93CF93DF93EC017F
:1001F000888111E08127888348DF82E0DCDF888105
:100200008127888342DFDF91CF911F913BCFA39A53
:1002100083E687B986EC86B93699FECF369A369949
:10022000FECFC5B1B99AB89A81EA8FBD81E083BF8C
:100230004ADF6ADFC63F80F080916C008F5F8F716C
:1002400080936C00809160008F5F8093600090913C
:1002500066008917D0F017C010926C00C53B78F08B
:100260008091600090916600891301C00CC08111DB
:1002700002C080916B0081508093600006C0809125
:100280006200811102C010926000FFDEBB9AC39A27
:10029000A29A81E687B986EC86B9369AC0E010E06A
:1002A0000FEF81EAF82E80916000E0916900F091F3
:1002B0006A00E80FF11DD49190916C00903160F0CC
:1002C000E1DE10926C001092600081E690E08CDF1D
:1002D00082E690E089DF44C0DD3F59F409BD16BED7
:1002E00082E390E0C6DEFFBC19BC16BE82E390E05C
:1002F00011C0DC3F89F4D4E009BD16BE85E090E072
:10030000B8DE19BC06BF81E490E0B3DED150A1F79E
:1003100080ED92E0AEDE24C0DE3F81F447DF982F0F
:1003200080E001C08F5FE82FF0E0EC5EFF4FE491CA
:10033000E917C0F340DFA6DEA5DE12C01FDF1F5F96
:100340001B3548F0DF3F39F480916600825080937E
:10035000600014DF9ADE84EF91E08BDE10926C0077
:10036000349BA1CF85B1813728F5CF5FC83018F114
:10037000C091600080916600C81798F4CC2311F0FA
:10038000C15010C0FFBC19BC16BE85B7877E806106
:1003900085BF85B7806285BF889585B78F7D85BF0E
:1003A00001C0C2E08C2FEADEC09360006EDE8AEFEF
:1003B00090E05FDEC0E0369A76CFE199FECF1FBABB
:1003C0008EBBE09A99278DB30895262FE199FECF31
:1003D0001CBA1FBA8EBB2DBB0FB6F894E29AE19AF5
:0A03E0000FBE01960895F894FFCFB8
:00000001FF
